:02000000B32823
:08000800FC000308FD00831257
:100010008C10A10B0E28C830A1003E158A012208C1
:100020008200051A68280830A3001830A20068284A
:10003000A30B6828051A66281230A3000830A40014
:10004000A5012430A2006828A30B68282D30051EC6
:100050003E30A2001230A3006828A30B6828051ABE
:100060003B280314A40DA50D1230A300243003185F
:100070004C30A20068286230A2006828A30B6828D0
:10008000051E66280310A40DA50D1230A300243010
:1000900003184C30A200682824083F39251E403838
:1000A000A40DA50DA40DA50DA40025081F39A800B9
:1000B0002408A9005E30A2003E14682862303E1C6D
:1000C000A20068281130051AA20068281130A20089
:1000D000A00AFF0133082002031C7F143408200209
:1000E000031CFF1435082002031C7F15360820026C
:1000F000031CFF1537082002031C7F163808200256
:10010000031CFF1639082002031C7F173A0820023F
:10011000031CFF177F0886007D088300FC0E7C0E01
:1001200009001F39820700340034013402340434DA
:10013000063409340C340F34133418341D3423348A
:1001400029342F3437343F34473450345A346434EC
:100150006F347A3486349334A034AE34BD34CC3426
:10016000DC34ED34FE3483018B018A018501860184
:1001700007309F008316FE308500003086008C011A
:1001800083120510203084008001840A7F3004022D
:10019000031DC4281130A200BE01A001AA012A300B
:1001A000840083169B018312093079216C2192010E
:1001B0008C0183167C3092008C1483120B178B17E2
:1001C000121505143E103E18F0283E19E828E328C1
:1001D0003E11BE1DE328BC0BE328BE110514E32825
:1001E000BE150530BC0005101030290603192D2955
:1001F00011302906031934290D30290603194F2916
:1002000001302906031975290230290603197529B9
:1002100003302906031975290430290603197529A5
:100220000530290603197529063029060319752991
:10023000073029060319752908302906031975297D
:100240000930290603193E290030290603193B29E4
:100250000C30290603194729E22842211F300006E5
:100260000319E228800A57294221003000060319A9
:10027000E2288003572942218001572942211F305B
:10028000800057292B3084002A08840708002A3070
:10029000840083169B01831209308421BE10BE1C8A
:1002A0005429BE106C21E228BE146C21E2282A08D1
:1002B0005A21E228BE18672984002B3084070008E1
:1002C0009120BD00083084073D08800008008400AC
:1002D0003330840780010800BB013B085A21BB0A68
:1002E00008303B06031D6D29080001302902AA00D1
:1002F000E228BD0083161C141A088000840A9B0A99
:100300008312BD0B7A290800BD0083161C158316C5
:1003100000089A0094219B0A840A8316BD0B872942
:1003200083161C11831208008B1355309D00AA30D0
:0C0330009D009C148B179C189B29080052
:02400E00623F0F
:10420000000005000500050005000000000000009A
:024210000000AC
:00000001FF
